:020000040000FA
:020000004A288C
:080008000B1D09000B11A10AF8
:1000100020083F3C031911282108F43C031D1A282D
:1000200017282108FD3C031D1A28A001A003A101E7
:10003000A00A2914AA010E1D2A148E1DAA140E1E30
:100040002A15B7010C1D371438083704031D2A2858
:10005000DF212B28DC21AB0A09008B1322008C0145
:100060008E0123008C018E012100833095001F300A
:100070008E0004308C002000FF308E00A001A10112
:10008000A401A301A201A901AA01AB01B8018B1629
:100090008B1708002D20FA207922BD227221B8206A
:1000A000291C5028E2210D221E22E9212C223D226A
:1000B000A910B820D42003198A28E221BC200319F2
:1000C0007128D821C420031D6828D42003198A2848
:1000D000291C6228A9183D22F0210D221E22A91CEC
:1000E0006228E2210D22E921BC2003195A28DA21D5
:1000F000C420031D7E28D42003198A28291C7828AF
:10010000A9181E22F0212C223D22A91C7828E921C1
:100110002C225A28DA21E2210D221E22E9212C224A
:100120003D22AD01E420D2212A189428CA200319C7
:100130004621CF2003191921C420031D9628D5215B
:10014000B221D420031DB6284E212A18A528CA2082
:10015000031DAC289E21DB20CF20031DB128962152
:10016000DE20C420031DA7282A1CB42809215228F8
:10017000A001A10129100800A208031D0800A3087E
:10018000031D0800A408080003112A1C0800031519
:10019000AB0108000311AA1C080003150800031195
:1001A0002A1D08000315080003112A1C0800E1207D
:1001B000031DD4280800AA18DB2808002A19DE2805
:1001C00008002B08823C0800EB20AC00AC19383E3C
:1001D000803EA82208008A012D08820700340134DD
:1001E0000334043406340734083409340B340C3433
:1001F0000E340F340030F0000030870030308600BD
:100200000730A5005C228100F00A4131A50B0229CC
:1002100008000030F00000308700303086000730E2
:10022000A5000108F1006522F00A4131A50B112952
:1002300008002C08403E860000308700810A2C0808
:10024000033C03192F292C08063C03192F292C08DD
:100250000B3C03192F292C080E3C031D34290108DF
:10026000363C031938293A2901083A3C031D3A293A
:10027000303081002C08AC19383E803EAE00A822F8
:1002800001089E222E08A822DE200800AD0A2D08B3
:100290000C3C0319AD01E420DB2008001030A50060
:1002A000A80100308700403086005E218100413186
:1002B000A80AA50B55291E223D22080001308A00FC
:1002C0002808820743346F346E34743472346134D6
:1002D000733474342034533465347434743469346E
:1002E0006E3467341030A500A8010030870040301C
:1002F0008600822181004131A80AA50B79291E229E
:100300003D22080001308A002808820749346E34F3
:10031000743465347234763461346C34203420346F
:100320002034543469346D346534723436083F3CBB
:10033000031DB60A3608B600A5210800B608031D3D
:10034000B6033608B600A52108003930A8223608C1
:100350000F397038A822360E03395438A8223830A5
:10036000A82208004030860000308700C621B00077
:100370004131C621B1004131C621B200C621B300CE
:100380004131C621B4004131C621B50016000F39F4
:10039000A800A8352808A835A835A80716000F39E1
:1003A000280708000F30A82208000C30A8220800F7
:1003B000381408003810080000308E000800203083
:1003C0008E0008003008A2003108A3003208A40003
:1003D00008003308A2003408A3003508A400080070
:1003E0002910A4032408031DFD292308031DFD294A
:1003F0002208031DFD29A91408002408FF3C031D41
:10040000042A3B30A400A3032308FF3C031D0B2A4E
:100410003B30A300A203A91008000030AC00220862
:100420004B223A30C2000330AC0023084B223A3052
:10043000C5000630AC0024084B2208008030A822FA
:100440000830A500403086000030870001089E2259
:100450004131A50B262A08000830AC0022084B22A7
:100460003A30CA000B30AC0023084B223A30CD00A2
:100470000E30AC0024084B220800C030A8220830FF
:10048000A500483086000030870001089E224131D7
:10049000A50B452A0800D000F22240302C07860028
:1004A00000308700520E0F39303E810052080F395C
:1004B000303E41318100080023007008910015137F
:1004C00095131514130820000800230070089100EC
:1004D000710893001513951315158B13553096005D
:1004E000AA30960095148B1715119518742A2000C0
:1004F0000800240095151511951015109417141364
:100500000930920095169513151320000800240059
:1005100016142000911D8A2A911108002400161536
:100520002000911D912A9111080024001418962A88
:1005300091002000911D9A2A91110800A80087229D
:100540007C30952240309522280895228E22080082
:10055000A80087227C309522003095222808952219
:100560008E22013028020319BB2A02302802031907
:10057000BB2AD8220800DE220800E622E622383014
:10058000A8223930A8221430A82236080F39703832
:10059000A822360E03395438A8226C30A822EC2247
:1005A000EC223830A8220D30A8220130A822080001
:1005B0000730A6000000A60BDB2A0800F830A600D2
:1005C0000000A60BE02AE42A000008001430A7006F
:1005D000DE22A70BE82A08006430A700DE22A70B62
:1005E000EE2A0800D101500E50070F398318163E2D
:1005F0008318063E063E831CFA3E501A1B3E831C9F
:10060000FA3ED01A303E501B603ED01B203E603E6A
:0E061000D10D511CA03ED200D01BD10A080013
:020000040001F9
:02000E00810F60
:02001000FF1ED1
:0EE000000000000005000000000005002000E8
:00000001FF
